:10100000F209F109D60AD50AD208D00824FF5021E6
:10101000FFFFFFFFFFFFFFFFFFFFFFFFFFFFFFFFE0
:1010200035200000008E2001BB00000003003DB20F
:10103000CA5800000000000000000000000000008E
:1010400000000000000000000000000000000000A0
:10105000008E268E2101FFFFFFFFFFFFFFFFFFFF36
:10106000FFFFFFFFFFFFFFFFFFFFFFFFFFFFFFFF90
:10107000FFFFFF003D9C09B1FF00000000000000E1
:10108000E62B021F8A0803010000E803E8030001C1
:1010900074990600FFFFFFFF00FFFFFFFFFFFFFF48
:1010A000FFFFFFFFFFFFFFFFFFFFFFFFFFFFFFFF50
:1010B000FFFFFFFFFFFFFFFFFFFFFFFFFFFFFFFF40
:1010C0009384FE16FFFFFFFFFFFFFFFFFFFFFFFF01
:1010D000FFFFFFFFFFFFFFFFFFFF08100080000082
:1010E0005F7FA30BBD0D757F01074408FE08FFFF5E
:1010F000FFFFFFFFFFFF0108B08FB28EA28D4A876E
:10E00000314000063C4066033D401E01B0125AFEFE
:10E01000B01266F4B012BAFE32C23140FE0532D2FE
:10E02000F240F30001033E4080100F43FF4E020315
:10E030001F533F900A00FA23F2400B0000033540C3
:10E040000003B012E8E7F240E1006804F240030088
:10E050006904B012F8E5B01238EBB0121AE6C24308
:10E060007404B0126EE6F29005007A041E34B2B069
:10E07000100062013F29B2B0100064012D28D2B314
:10E080000100F12FF29003001F040C38B0128AEC4B
:10E09000B01278E3F2900A0074040438B01220FC45
:10E0A000B01278E3B0126EE6DE3FF240F4000103F6
:10E0B0003E4080100F43FF4E02031F533F900A0063
:10E0C000FA23F2400B00000335400003B012E8E7EA
:10E0D000D2C31900E2C32900B01270FAC43F3FF066
:10E0E0003F003F50A00F12C30F10F0400700BA22AC
:10E0F000C04FB5223F4010002B433C40A703B01255
:10E10000F2E6C23D0F43FF4E01031F535F9200032F
:10E11000FA233041B0128CE3B012FCEAA2C36001D2
:10E12000D24276033F03D24277034003F2D080000D
:10E130004003F2D020004003D2426D043E030E4360
:10E140005E426D04A2D360010E5E0E5ED24E0010E0
:10E1500041031E53D24E001042031E53D24E0010F4
:10E1600043031E53D24E00104403B0126EE9B012A6
:10E17000B4E9B012C2E9C24E48038E10C24E490340
:10E18000B01220E9B012B4E9B012C2E90E110E11BA
:10E19000C24E45038E10C24E4603B012D4E8B012F0
:10E1A000B4E9B012C2E90E110E110E110E11C24ED9
:10E1B0004703B0123AE9B012B4E9B012C2E9C24E54
:10E1C0004C038E10C24E4D03B012BCE8B012B4E93D
:10E1D000B012C2E9C24E55038E10C24E5603B012A1
:10E1E000A4E8B012B4E9B012C2E9C24E57038E10CF
:10E1F000C24E5803B012EEE8B012B4E9B012C2E950
:10E20000C24E4E038E10C24E4F03B01208E9B01238
:10E21000B4E9B012C2E9C24E59038E10C24E5A037D
:10E22000A2C36001C2436F04D2437004A2D3600151
:10E23000B2900F006C031B2CB2B010008401F82FB9
:10E24000B2900E0072032634B2900D0072030520C6
:10E25000B29021DF70031E34003CD24270033503BC
:10E26000D24271033603D24272033703213CB2B06B
:10E27000100084011928B2C01000840182936E033B
:10E280000920B2437003B240FF007203B2C0100015
:10E290008401E33FB24021DF7003B2400D007203FE
:10E2A000B2C010008401D93FB2C010008401D53F34
:10E2B000D240C22D3203D240BD2D3303D240B82DFF
:10E2C0003403D240B42D3803D240AF2D3903D240AD
:10E2D000A72D3A03D040AA2D8820D040A52D832019
:10E2E000D040A02D7920D0409C2D7520D040952D78
:10E2F0006E203041D24266046504B012A0FEF2D016
:10E3000080007004D2C30100E2C31900F2C02000F3
:10E310003300F2C020003200D2C31F00D2C31E005F
:10E32000F2C020002A00F2C22A00F2C010002A0027
:10E33000F240E1006804C2436904B012F8E5F290CB
:10E3400005007A043634B2B010006201F82FF29062
:10E350000300A303CF27F2906200A3032E24F290C0
:10E360006100A3035024F2906000A3037A24F2908A
:10E370005700A3038924C33FB01214E1D2426404BE
:10E38000000335400003B012E8E73041A2D360013A
:10E39000034303430343034303430343A2C3600113
:10E3A000A2B3A001F32FF2D080007004A2D36001C9
:10E3B0003041D2C31900E2C329000B430C430F4381
:10E3C0005B42A6034B939B273B902100982F5F4213
:10E3D000A5033F908000932F0C4F0C5B3C90810075
:10E3E0008E2F3C40A703F2900A00A4030824F29069
:10E3F0000B00A4038423B012FEE6053C803FB0125C
:10E40000F2E6013C7C3F0B430C430F435B42A60307
:10E410004B9375273B908100722F5F42A5033F907D
:10E4200080006D2F0C4F0C5B3C908100682FF290A8
:10E430000A00A4030724F2900B00A40360233D40CC
:10E440000010023C3D4080100D5FB012ACFEF24067
:10E4500005006504B012A2FCB012ACE5B012ECFDF0
:10E460004E3FD2437004B01214E1B012ACFEE2434E
:10E470006504B012A2FC3D4032037B403100B01273
:10E48000ACE5B012ECFD3B3FD2D30100F2D020004E
:10E490003300F2D020003200D2D31F00D2D31E00AE
:10E4A000F2D020002A00F2D22A00F2D010002A0076
:10E4B000E2D31900B240B4DC9E038243A003B01241
:10E4C00004FED24370043B41B012B2FB3B4010004B
:10E4D0000E6EB012EAE41B83FB233B4010000C6C71
:10E4E000B012EAE41B83FB23273C0428F2D010007F
:10E4F0002900033CF2C010002900034303430343F7
:10E50000034303430343F2D02000290003430343A2
:10E5100003430343034303430343034303430343CB
:10E5200003430343F2C02000290003430343034392
:10E530000343034303433041034303430343034380
:10E5400003430343F2D2290003430343034303433A
:10E55000034303430343034303430343034303438B
:10E56000F2C229000343034303430343034303432A
:10E570003041F2C020002900F2C229003E4044038D
:10E580001C408C2AB012CCE41C40FC1E1E40FA1E1B
:10E59000B012CCE40E433C40E25FB012CCE43E400B
:10E5A00074003C40AF18B012CCE430410C43F04D45
:10E5B000B61DF0901000B01D0520B012D0E5F0405F
:10E5C0001000A41DB012D0E51C530B9CF023304169
:10E5D000D2436B04B2400900680312127001B150BB
:10E5E000A0010000B2417201B240B0006201B2B0BD
:10E5F00010006201FC233041C2436604D2C36704A9
:10E60000E2C3670482436A03C2436B04B240090059
:10E610006803B240149162013041D2C30100F2405C
:10E62000D0006200C2436300F24006006400F2D0F2
:10E6300020001000F2D030001B00C2436000F24006
:10E64000800061003041D2C30100F24082006200CC
:10E65000F24006006300F24006006400F2D0300091
:10E660001B00C2436000F240800061003041D2C311
:10E670000100C243650080430C1ED2D3010030412B
:10E68000E2B30300FD2BD240F01C67003041F040A4
:10E690001000E61CB01280E6F89010000000052083
:10E6A000F0401000D41CB01280E6F048CC1CB01230
:10E6B00080E6D083BD1DF023F0401000BC1CB012DA
:10E6C00080E6F0400300B21CB01280E630413F40CB
:10E6D00010002B433C40A703B012F2E630413F400C
:10E6E0000F001B43D243A7033C40A703B012F2E63E
:10E6F00030413F90400009343D4080100F3C3F9036
:10E70000400008343D400010093C3F8040003D403F
:10E710004010043C3F8040003D40401032C20D128A
:10E72000B0123EE72D41B0127CE7FF4CDE031F53D1
:10E730001B83FB233D41B01250E732D230410E43E0
:10E74000AE4DDE032D532E533E904000F923304151
:10E75000B04000A5D819B04040A5CE190E439D4E3B
:10E76000DE0300002D532E533E904000F823B040AE
:10E7700000A5B619B04010A5B4193041B24000A5AB
:10E780002C0192B32C01FD2FB24002A52801CD43EC
:10E79000000092B32C01FD2FB24010A52C01304196
:10E7A00005120B430E435E4200035E830D437D451D
:10E7B0003F421DB3013C4D6D0C6C0B120B100CEB6A
:10E7C0000B100B100CEB0B100B100CEB2B410B6B0D
:10E7D0000B6B0B6B0CEB3B410C100B6B1F83EB2398
:10E7E0001E83E42335413041F2C080006203D253DE
:10E7F0006203F290650062030228D2436203B2D042
:10E80000800062030F3CD292640400030B24F29058
:10E81000470001030720D25300035F420003DF4299
:10E8200062030103D2D31F00F2D080002900B0128E
:10E8300018EBE2436C04C2936C04FD23E253000323
:10E84000B012A0E70F435F420003CF4B00031F83CA
:10E850008B10CF4B0003D242000365045B420003E0
:10E86000F24080007604B0401000101B0D451D538F
:10E87000B012ACFEF040E200EE1AB012D0E5F0406B
:10E880005500E41AB012D0E5D0426504DA1AB0128D
:10E89000D0E5B012ACE5B012ECFDB0902200DC1A6D
:10E8A000FC233041A2C3A0018243A4014D43B240E6
:10E8B000F00FA001B240F202A201663CA2C3A00187
:10E8C0008243A4015D43B240F00FA001B240F202C6
:10E8D000A2015A3CA2C3A0018243A4017D401200C0
:10E8E000B240F00FA001B240F202A2014D3CA2C31F
:10E8F000A0018243A4017D400300B240F00FA001BB
:10E90000B240F202A201403CA2C3A0018243A40192
:10E910006D42B240F00FA001B240F202A201343CBD
:10E92000A2C3A0018243A4017D401500B240F00FB4
:10E93000A001B240F202A201273CA2C3A00182437F
:10E94000A4017D401600B240F00FA001B240F202D7
:10E95000A2011A3CA2C3A0018243A4017D4007008A
:10E96000B240F00FA001B240F202A2010D3CA2C3DE
:10E97000A0018243A4017D401A00B240B00FA00163
:10E98000B240F202A201003CC24D8000C24D8100A3
:10E99000C24D8200C24D8300C24D84007DD08000F4
:10E9A000C24D8500034303430343A2D3A00192D386
:10E9B000A0013041B2B02000A401FC2BA2C3A001F1
:10E9C00030413F4040010E4F0D4F2F532C4F2C9E96
:10E9D00001380E4F2C9D01340D4F3F904A01F52315
:10E9E0000E9D01202E538E4300008D4300003F40BA
:10E9F00040012E4F2F532E5F3F904A01FB230E11F3
:10EA00000E113041331291830000FD232153304118
:10EA1000B240805A2001E2D32200E2D32600F0C0A7
:10EA20001800FF15F0D0E000F915E2D22600E2D27E
:10EA30002E00F240BA002A00F2C020002900F2C2E3
:10EA40002900F2D010002900E2C32900D2D31A0015
:10EA5000E2D21A00E2D31A00D2C31900E2C21900AE
:10EA6000E2C31900F24009001E00D2D31F00E2D316
:10EA70001F00F2D020003200F2D020003300F2D08C
:10EA800040003200F2D040003100F2D0800032006D
:10EA9000F2C080003100F2C23300F2D23200F2C282
:10EAA0003100F24337003041F2C080005700F2D00D
:10EAB00080005300F2D020005300E2C302003F4028
:10EAC000FF471F83FE23E2B30200F723B01204EADC
:10EAD000F240880058003041A2426201B240240056
:10EAE0006201B24062026001304182436C03B24075
:10EAF00046028001B2D020008001304132C2824300
:10EB00006C03824370038243720382436E03B240FC
:10EB10001041840132D2304182436C0312129001C1
:10EB2000B15040030000B2419201B04022004C18A5
:10EB3000B240900082013041C2437704B0423E1897
:10EB4000B240308164013041F2457604A0532C1864
:10EB5000B0F00F0026180B20C29300030620F242EB
:10EB60000003B04024001418023CD2830003D252A8
:10EB700076047604182CB250400392013041B25012
:10EB800040039201D28300030D20B0402200EC1715
:10EB9000B2C010008201F2C080002900D2C31F0061
:10EBA000D2C31D003041B250A001920190D3CC17C6
:10EBB0003041B250A001920190C3C0173041B0F073
:10EBC0001F00B8170224A053B217D252760476045D
:10EBD000EA2FB250400392013041B250A00192019D
:10EBE000A0539817304110521E013041083C30416B
:10EBF000304130413041304192536C033041A2B337
:10EC000084010B28B2C010008401A2C38401824396
:10EC10007203B2400F007003304182936E030920EB
:10EC200092429401700392426C03720392536E03FA
:10EC30003041929056246E032338B2C010008401F4
:10EC4000A2C3840112126C03918272030000B241CC
:10EC5000720392B38001826372030820121294013E
:10EC6000918270030000B2417003304192837203BD
:10EC7000B2E37003925294017003826372033041D5
:10EC80008293940192536E0330410A120B120812C0
:10EC9000091206120712D2537404D24236048A03B0
:10ECA000D24235048B03D24234048203D24233046D
:10ECB0008303D24232048403C2438503D242240434
:10ECC0008C03D24223048D03D24222048E03D2420B
:10ECD00021048F03D24228049003D24227049103D7
:10ECE000D24226049203D24225049303C2439403E2
:10ECF000D2422B049503D2422A049603D24229041D
:10ED00009703D2422D049803D2422C049903D24295
:10ED10002F049A03D2422E049B03D24231049C0357
:10ED2000D24230049D03B29095038A03042CB25062
:10ED300000088A03033CB25000048A035E42370491
:10ED40004E4E0F431E5282031F6284033A40E80373
:10ED50000B43021232C20343824E3001824A380111
:10ED6000824E340192423A01860392423C013A01BA
:10ED7000824B3801824F3401824A380192423A0173
:10ED800088033241B2900C2488030D380420B290DD
:10ED9000008486030828B250007C8603B260F3DB4F
:10EDA000880392538A033840804A39405D050A43FC
:10EDB0000B431C428C031D428E030E4D3EE30E5E40
:10EDC0000E7E0F4EB012DEFCB012DEFC0F4E0E4D6A
:10EDD0000D4C0C43B012C2F8824C8C03824D8E0352
:10EDE000384000953940BA0A0A430B431C4290034D
:10EDF0001D4292030E4D3EE30E5E0E7E0F4E0E1030
:10EE00000F4D0F100E4C0E100D430D100C43B01291
:10EE1000C2F8824C9003824D92031C4294031D421F
:10EE200096033E4000010F43B01262FC824C9403F3
:10EE3000824D96031E4294031F4296030E5E0F6F8F
:10EE40000A4E0B4F0E5E0F6F0E5E0F6F0E5A0F6B5A
:10EE5000824E9403824F9603B29001C098031438F7
:10EE6000B290004098031034B29001C09A030C385D
:10EE7000B29000409A030834B29001C09C03043859
:10EE8000B29000409C031838D2437E041C42980381
:10EE90002E43B01254FD824C98031C429A032E4319
:10EEA000B01254FD824C9A031C429C032E43B012B4
:10EEB00054FD824C9C03113CC2437E041F429803C4
:10EEC0000F5F824F98031F429A030F5F824F9A038E
:10EED0001F429C030F5F824F9C03C24380044F4339
:10EEE0007F900C00082C4F4FCF9348040224D2533C
:10EEF00080045F53F53F5E4220046E8303245E83EB
:10EF00000824163CE2421D03C2437F04C243750439
:10EF1000163CC2431D03F29003007504032CD25328
:10EF20007504023CE2437A04D24280047F04073C29
:10EF3000F24005001D03C2437F04C2437504F24042
:10EF40009F000103F24020000203C2430303D242A8
:10EF500099030403D24298030503D2429B0306039C
:10EF6000D2429A030703D2429D030803D2429C0374
:10EF70000903D24289030A03D24288030B03D24217
:10EF800087030C03D24286030D03D2428F030E0384
:10EF9000D2428E030F03D2428D031003D2428C0360
:10EFA0001103D24293031203D24292031303D242BB
:10EFB00091031403D24290031503D2429703160320
:10EFC000D24296031703D24295031803D242940308
:10EFD0001903D2427E041A03C2431B03C2431C031B
:10EFE000D2427F041E03D24237041F03D2428B0356
:10EFF0002003D2428A032103D242480422034F4312
:10F000007F900C00072C4B4F4F4FDF4B48042203DF
:10F010005F53F63F1C4294031D4296033E40E803B3
:10F020000F43B01262FC064C074DC2937A1028249D
:10F03000F2937A100320F2D23100223C021232C243
:10F040000343D2427A103001B240E80338011F4234
:10F050003A0132410B4F0E4B0F430F9703380E20EE
:10F060000E960C2C0E4B3E50F4010F43079F0338B5
:10F070000520069E032CF2D23100023CF2C2310080
:10F08000C2934A0315200793113803203690891341
:10F090000D28F2900A007D040620B012DEE6D2426E
:10F0A0008F104A03053CD2537D04023CC2437D04C9
:10F0B000304082FE0A120B120D120C120F120E12A9
:10F0C00010522E01C93D043CC73DC63DC53D403CE4
:10F0D00032C0D00092527E037401B2B000106401BD
:10F0E000162882937C030420B2C010006401B43D52
:10F0F000B2D080006401D2B377040328B2C080008C
:10F10000640112C352107704B2537C03A53DB2B020
:10F11000000164010A28B2C0000164011E427E039E
:10F1200012C30E10825E7401973D12C35210770411
:10F13000B2B0000464010328F2D080007704B25317
:10F140007C0382937C038821B2C010006401843D5B
:10F15000F2905C007B04032CD2537B04023CC2433C
:10F160007B045E427A044E8338245E8307245E83E8
:10F1700066245E8319245E833024763C5E427B04E1
:10F180005E8307247E801E0008247E803C000924C4
:10F190006B3CF2D080003100673CF2C0800031004F
:10F1A000633CC2437B04603C5E427B045E830A2472
:10F1B0005E830C245E8306245E8308247E801B000D
:10F1C0000924523CF2D0800031004E3CF2C0800055
:10F1D00031004A3CC2437B04473CB290C1117E03DC
:10F1E00016205E427B045E8305246E8207246E82B5
:10F1F00009243A3CF2D080003100363CF2C0800055
:10F200003100323CC2437B04D2537C042D3C5E422D
:10F210007B045E8307247E801E0008247E801E00FF
:10F220000924223CF2D0800031001E3CF2C0800054
:10F2300031001A3CC2437B04D2537C04153C5E422D
:10F240007B045E8307247E80050008247E801900ED
:10F2500009240A3CF2D080003100063CF2C0800054
:10F260003100023CC2437B04C2937A042F24D2B300
:10F270002800142CD2937C040428F2D080003100A2
:10F28000253CE2427A04B290C1117E031F20F29025
:10F290000A007B041B28C2437B04183CD2937C04E5
:10F2A0000428F24005007A04113CC2937C040E2429
:10F2B000C2437C04C2437B04B290C1117E0304208C
:10F2C000F24003007A04023CD2437A04C2936C04F5
:10F2D0000224F2536C04C29379040324F253790498
:10F2E000023CC2437804C2937004B638C2936E04E1
:10F2F0000520D2436E04B012D2FBAE3CC293700420
:10F300008320B2B02000A401A728A2C3A0014D43CE
:10F310003C40FF0F4F437F9006000C2C4E4F0E5E7B
:10F320001C9E400105284B4F0B5B1C4B40014D4F71
:10F330005F53F13F4B4D0B5B8B4340014D430C43FF
:10F340004F437F9006000C2C4B4F0B5B1C9B4001E6
:10F35000052C4B4F0B5B1C4B40014D4F5F53F13F56
:10F360004B4D0B5B8B434001824376034F437F90B1
:10F370000600072C4B4F0B5B925B400176035F53FB
:10F38000F63F12C31210760312117603D2426E04B6
:10F390006F045E426E045E8305245E8307245E83F1
:10F3A0000A240D3C0C433A40B80B093C3C4078051C
:10F3B0003A401C0C043C3C4020033A40FF0F829C26
:10F3C0007603082CE2936E041028F2536E04B012F8
:10F3D000D2FB0B3C1A927603082CF29003006E04C9
:10F3E000042CD2536E04B012D2FBD24370045E429E
:10F3F0006F047E53C24E6D04F29003006E042C2005
:10F40000F2D080007004283CF2537004C293700460
:10F410002320A2C3A0018243A401B240F00FA001A7
:10F42000B240F202A201F24007008000F240070061
:10F430008100F24007008200F24007008300F240A2
:10F4400007008400F2408700850003430343034321
:10F45000A2D3A00192D3A0013E413F413C413D4196
:10F460003B413A410013B2B040002C010328B240A6
:10F4700040A52C01C2430003C2430103C24332032F
:10F48000C2433303C2433403C2433503C24336038A
:10F49000C2433703C2433803C2433903C2433A036A
:10F4A000D2420C103B03C2433C03C2433D03C24360
:10F4B0003E03C2433F03C2434003C2434103C2432E
:10F4C0004203C2434303C2434403C2434503C2430E
:10F4D0004603C2434703C2434803C2434903D242DF
:10F4E0008F104A03D24298104B03C2434C03C243CD
:10F4F0004D03C2434E03C2434F03F2922410032034
:10F50000D2435003023CC2435003C2435103C2439F
:10F510005203C2435303C2435403C2435503C2437D
:10F520005603C2435703C2435803C2435903C2435D
:10F530005A03F2435B03C2435C03C2435D03C2430D
:10F540005E03C2435F03C2436003C2436103C2431D
:10F550006203C2436303F24062006404C243DE03F9
:10F5600082436C0382436E038243700382437203BF
:10F5700082437403C2437104C2437304C2437404DC
:10F58000C2437504C2437604C2437D0432C20343BE
:10F59000F24080007004C2436604C2436704B012A4
:10F5A00010EAB2400C8E7E03B012A8EAB012D8EA7C
:10F5B000B012EAEAB0121CFEB01238EB32D2C243EB
:10F5C0007A04D2437C04C29373101A20E2B21C0066
:10F5D000172CD2D319003E40204E0F430D4E0DDFA5
:10F5E0000D9303243E533F63F93FE2D21900E2D367
:10F5F0001900F2D080003100D2437A04B012B2FB7D
:10F60000D2D31900E2C21900E2C31900D2B3280014
:10F61000FD2BD2937C040E28F2D080003100E2D280
:10F620001900E2D31900C2437C04D2437A04B01219
:10F63000B2FB023CD2C319001C4330410F12B2503E
:10F64000A0017201C2936B042324929368030620E5
:10F65000B2C080006201B2536803BD3C829368036C
:10F660000720B2C010006201B2C080006201B33C4A
:10F6700092B366030428B2C080006201033CB2D09A
:10F680008000620112C312106603B2536803A33CE8
:10F69000B290090068030920B2C000016201B250B3
:10F6A000D0007201B2536803963C8293680314241D
:10F6B000B2B0000462010428B2D080006603033CAB
:10F6C000B2C08000660392936803032412C3121031
:10F6D0006603B25368037F3CB2D014816201B2402A
:10F6E0000900680382936A031F201F4266033F805C
:10F6F00003000C243F800D000F20C2936A040324F2
:10F70000C2436A04683CD2436A04653CC2936A04FB
:10F710006224C2436A045F3CD2426603A20392435E
:10F720006A03C2436A04573CB29063006A03512CD7
:10F730001F4266033F80030013243F800D003F20DB
:10F74000C2936A040A24C2436A041F426A03DF4266
:10F750006603A20392536A033E3CD2436A043B3CD5
:10F76000C2936A042424C2436A04D2426A03660430
:10F77000C29368041924D292A20368041520C2938C
:10F7800069040420B2C010006201253CC2936904E0
:10F790000824D292A30369040420B2C010006201BD
:10F7A0001A3C82436A03173C82436A03143C1F429B
:10F7B0006A03DF426603A20392536A030C3CC2430E
:10F7C0006A041F426A03DF426603A20392536A037C
:10F7D000023C82436A033F41001306930224B012A5
:10F7E0006CFE3641304106120B120A120912081241
:10F7F00031801000814C0800814D0A00814E0C00C0
:10F80000814F0E00814300008143020081430400C8
:10F8100081430600B0128AF8B012A8F8B1B0008097
:10F820000E00B01298F891510800080091610A008A
:10F830000A0091610C000C0091610E000E001F91F6
:10F84000160016280B201E911400122807201D9167
:10F8500012000E2803201C9110000A281C811000A1
:10F860001D7112001E7114001F71160091D300004B
:10F870007653D2232C411D4102001E4104001F413A
:10F88000060031501800364130410C430D430E4301
:10F890000F43764040003041087818530C5C0D6DE2
:10F8A0000E6E0F6F0CD83041915102000200916131
:10F8B0000400040091610600060091610800080040
:10F8C00030410612B01290FE0334B01248FE16E327
:10F8D000B012E6F7823FE2C21900E2C31900F2F06B
:10F8E00003002200F2C020002900F2C22900F2C069
:10F8F00010002900F2C080002900F2C010001B0097
:10F90000F2C010001900F2C020003300F2C0200045
:10F910003100F2C040003100E2D32900D2C3190007
:10F92000B01238EBF24003007A04C2437B04D242A7
:10F93000FE105600D242FF105700C2435800F2405A
:10F9400020005300B240C1117E03F2C0800031009C
:10F95000F29005007A040520D2C31900E2C3290001
:10F96000FF3FB2B010006401F32FB01270FA4C9355
:10F97000EF27B01210EAD2436E04B012D2FBF2D0DD
:10F9800010001B00D2D319003E40204E0F430D4EF5
:10F990000DDF0D9303243E533F63F93FE2D319007B
:10F9A000E2D21900E2C32900B012B2FD3040B2FB2E
:10F9B0000F12E2B265000428F2F083006500563CA5
:10F9C000F290AA0066002D20E29381040D20C2432C
:10F9D0008104D24382045F4284044F4FDF426600B9
:10F9E0001E04D2538404423CC293820417245F4213
:10F9F00084044F4FDF4266001E045F4284044F4F71
:10FA0000FF90AA001E040720D29384040420F24031
:10FA1000AB001E042B3CD2538404283CD2538104F7
:10FA2000253CC29382042024F2903A0084041328D7
:10FA30005F4284044F4FDF4266001E04D2538404A9
:10FA4000C2438204D24284047204F240270072044A
:10FA5000D2C301000B3C5F4284044F4FDF4266007B
:10FA60001E04D2538404023CC24381043F4100136C
:10FA70000A124A43C29377044A24C24378045E427E
:10FA800077047E80410007247E800C0007247E805E
:10FA900005000624083CB012D6F8393C5A43373CDE
:10FAA000B012B2FB343CF290810077043028F2901F
:10FAB000BD0077042C2CF29003007A042320B012AE
:10FAC00010EAD2436E04B012D2FBF2D010001B0039
:10FAD000F2D020003300D2D31900E2C329003E4007
:10FAE000A0861F430D4E0DDF0D9303243E533F634D
:10FAF000F93FE2D21900E2D31900B012A8EAB240ED
:10FB00000C8E7E035C427704B01284FD5A43B0121F
:10FB100038EB4C4A3A4130410D120C120F120E12C2
:10FB200092B37A030328B012B2EB3E3C1F427A0331
:10FB30003F902500392C0F5F104F3CFB86FBA8FB44
:10FB40008CFBA8FB8CFBA8FB8CFBA8FB8CFBA8FB0D
:10FB50008CFBA8FB8CFBA8FB8CFBA8FB92FBA8FBF7
:10FB600098FBA8FB92FBA8FB92FBA8FB92FBA8FBCF
:10FB700098FBA8FB92FBA8FB92FBA8FB92FBA8FBBF
:10FB80009EFBA8FBA4FBB01248EB0E3CB0124CEB62
:10FB90000B3CB012BEEB083CB012DAEB053CB012E5
:10FBA00076EB023CB0127EEB3E413F413C413D4191
:10FBB0000013B012F8FEB01272E5D2B32000FD2B94
:10FBC000D2428F104A03D2420C103B0332D2304053
:10FBD00018E05E426E045E8305245E830C245E831F
:10FBE00013241A3C5E4222007EF003007ED0800087
:10FBF000C24E2200113C5E4222007EF003007ED005
:10FC00005000C24E2200083C5E4222007EF00300FB
:10FC10007ED02800C24E2200F24005007004304120
:10FC20000A12C2437404F24049000103D242800424
:10FC300002034A437A900C00122C4A4A4F4A0F5F43
:10FC4000DF4A480403034A4A5C4A38046E42B01251
:10FC5000D0FD4F4A0F5FCF4C04035A53EB3F3A415C
:10FC60003041091209430F9305343EE33FE31E532D
:10FC70000F6319D30D9305343CE33DE31C530D632F
:10FC800039E3B01218FD19B304243CE33DE31C53DF
:10FC90000D6329B304243EE33FE31E530F63394150
:10FCA00030410A12F240E200A2030A43C293650403
:10FCB0001424FA901000A2030520B240100066033D
:10FCC000B012D0E55F4AA2034F4F824F6603B012D5
:10FCD000D0E5F25365041A53E93F3A4130410C5CD8
:10FCE0000D6D0E6E0F6F0C5C0D6D0E6E0F6F0C5C5C
:10FCF0000D6D0E6E0F6F0C5C0D6D0E6E0F6F0C5C4C
:10FD00000D6D0E6E0F6F0C5C0D6D0E6E0F6F0C5C3B
:10FD10000D6D0E6E0F6F304109120A120B120A435D
:10FD20000B43394020000C5C0D6D0A6A0B6B0A8E88
:10FD30000B7F04281CD33953F623043C0A5E0B6F57
:10FD40003953F1230E4A0F4B3B413A41394130417F
:10FD50008C118E11091209430E9303343EE31E5396
:10FD600019D30C9303343CE31C5339E3B012D4FD94
:10FD700019B302243CE31C5329B302243EE31E536F
:10FD8000394130410A1221834A4C4C4A3C50200FE1
:10FD90002E43B01254FD814C0000D2410100A80353
:10FDA000E241A703B012CEE6B012B2FB21533A41B2
:10FDB0003041D2437A04D2D31900E2C32900E2D2FF
:10FDC0001900E2D31900B2400C8E7E033040A8EA3D
:10FDD0007CF37EF30F4E0D4C0E431C430D5D0E6EF7
:10FDE0000E9F01280E8F0C6CF92B3041B240100091
:10FDF0006603B012D0E5B24003006603B012D0E54E
:10FE00003040F8E51E429E031F42A0030D4E0DDF59
:10FE10000D9303243E533F63F93F3041C2436D04C9
:10FE200082437603C2436E04C2436F04D24370041C
:10FE300030410D120C120F120E12B012E6EB3E41C1
:10FE40003F413C413D41001338E339E33AE33BE3B2
:10FE5000185309630A630B6330410F4C0F5D033C79
:10FE6000CC4300001C530C9FFB2330413CE33DE39B
:10FE70003EE33FE31C530D630E630F633041354196
:10FE8000344137413641394138413B413A413041B3
:10FE900006430F930334B0126CFE16430B933041AC
:10FEA000B012ACFEB012A2FC3040ECFDB24010002B
:10FEB00066033040D0E53040BEFE3040B6FEFF3F26
:10FEC00009120A120B120A430B43394020000C5C42
:10FED0000D6D0A6A0B6B0A8E0B7F04281CD33953F5
:10FEE000F623043C0A5E0B6F3953F1230E4A0F4B85
:10FEF0003B413A41394130415C4290108C101D42E7
:10FF000092108D105A4291100DEA0F433E40F401B9
:10FF1000B012C0FE0C5C0D6D0C5C0D6D1C53804C62
:0CFF20006605804D64053041FFFFFFFFC7
:10FFE000FFFFFFFFFFFFFFFFFFFFFFFFFFFFB0F976
:10FFF000B4F03CF6FFFFFFFF32FE18FBFFFF00E00E
:00000001FF
